 esdhc

 Timestamp is 4da293b0 (Mon Apr 11 17:37:52 2011)

 Preferred load address is 10000000

 Start         Length     Name                   Class
 0001:00000000 0000019cH .rdata                  CODE
 0001:0000019c 00000022H .rdata$debug            CODE
 0001:000001c0 00005440H .text                   CODE
 0001:00005600 0000003cH .xdata                  CODE
 0001:0000563c 00000050H .idata$2                CODE
 0001:0000568c 00000014H .idata$3                CODE
 0001:000056a0 000000f4H .idata$4                CODE
 0001:00005794 00000104H .idata$6                CODE
 0001:000058a0 000000c7H .edata                  CODE
 0002:00000000 000000f4H .idata$5                DATA
 0002:000000f4 0000004cH .data                   DATA
 0002:00000140 00000040H .bss                    DATA
 0003:00000000 000003c8H .pdata                  DATA

  Address         Publics by Value              Rva+Base       Lib:Object

 0000:00000000       ___safe_se_handler_table   00000000     <absolute>
 0000:00000000       ___safe_se_handler_count   00000000     <absolute>
 0001:0000001c       ??_C@_1CC@LMBBBPNF@?$AAR?$AAe?$AAa?$AAd?$AAW?$AAr?$AAi?$AAt?$AAe?$AAT?$AAi?$AAm?$AAe?$AAo?$AAu?$AAt?$AA?$AA@ 1000101c     bspesdhc.obj
 0001:00000040       ??_C@_1BM@NNIPIGOJ@?$AAW?$AAa?$AAk?$AAe?$AAu?$AAp?$AAS?$AAo?$AAu?$AAr?$AAc?$AAe?$AAs?$AA?$AA@ 10001040     bspesdhc.obj
 0001:0000005c       ??_C@_1BG@OINKPJMJ@?$AAD?$AAi?$AAs?$AAa?$AAb?$AAl?$AAe?$AAD?$AAM?$AAA?$AA?$AA@ 1000105c     bspesdhc.obj
 0001:00000074       ??_C@_1BK@KBGNDCFC@?$AAS?$AAD?$AAI?$AAO?$AAP?$AAr?$AAi?$AAo?$AAr?$AAi?$AAt?$AAy?$AA?$AA@ 10001074     bspesdhc.obj
 0001:00000090       ??_C@_1CM@FPPMGDBH@?$AAM?$AAa?$AAx?$AAi?$AAm?$AAu?$AAm?$AAC?$AAl?$AAo?$AAc?$AAk?$AAF?$AAr?$AAe?$AAq?$AAu?$AAe?$AAn?$AAc?$AAy?$AA?$AA@ 10001090     bspesdhc.obj
 0001:000000bc       ??_C@_1M@EENNDIOJ@?$AAI?$AAn?$AAd?$AAe?$AAx?$AA?$AA@ 100010bc     bspesdhc.obj
 0001:000000c8       ??_7CESDHCBaseEDMA@@6B@    100010c8     bspesdhcdma.obj
 0001:000000e4       ??_7CESDHCBaseSDMA@@6B@    100010e4     esdhcbase_common_topaz_v1:esdhc.obj
 0001:00000100       ??_C@_1CC@NMDOMPHL@?$AAM?$AAS?$AAC?$AA_?$AAD?$AAE?$AAT?$AAA?$AAC?$AAH?$AA_?$AAE?$AAV?$AAE?$AAN?$AAT?$AA?$AA@ 10001100     esdhcbase_common_topaz_v1:esdhc.obj
 0001:00000124       ??_C@_1BG@MPOEBAN@?$AAM?$AAS?$AAC?$AA_?$AAS?$AAD?$AAD?$AAI?$AAS?$AAK?$AA?$AA@ 10001124     esdhcbase_common_topaz_v1:esdhc.obj
 0001:0000013c       ??_C@_1M@LJLEHHPO@?$AAE?$AAS?$AAD?$AAH?$AAC?$AA?$AA@ 1000113c     esdhcbase_common_topaz_v1:esdhc.obj
 0001:00000148       ??_7CESDHCBaseDMA@@6B@     10001148     esdhcbase_common_topaz_v1:esdhcdma.obj
 0001:00000164       ??_7CESDHCBase32BitADMA@@6B@ 10001164     esdhcbase_common_topaz_v1:esdhcdma.obj
 0001:00000180       ??_7CESDHCBase32BitADMA2@@6B@ 10001180     esdhcbase_common_topaz_v1:esdhcdma.obj
 0001:000001c0       ?ValueDW@CReg@@QAAKPBGK@Z  100011c0 f i bspesdhc.obj
 0001:0000020c       ?BspESDHCGetBaseClk@CESDHCBase@@QAAKXZ 1000120c f   bspesdhc.obj
 0001:00000250       ?BspESDHCInit@CESDHCBase@@QAAHXZ 10001250 f   bspesdhc.obj
 0001:00000604       ?BspESDHCDeinit@CESDHCBase@@QAAXXZ 10001604 f   bspesdhc.obj
 0001:00000608       ?BspESDHCSysIntrSetup@CESDHCBase@@QAAHXZ 10001608 f   bspesdhc.obj
 0001:000006bc       ?BspESDHCSetClockGating@CESDHCBase@@QAAXK@Z 100016bc f   bspesdhc.obj
 0001:00000760       ?BspESDHCSetSlotVoltage@CESDHCBase@@QAAXK@Z 10001760 f   bspesdhc.obj
 0001:00000764       ?BspESDHCIsCardPresent@CESDHCBase@@QAAHXZ 10001764 f   bspesdhc.obj
 0001:00000820       ?BspESDHCSlotStatusChanged@CESDHCBase@@QAAHXZ 10001820 f   bspesdhc.obj
 0001:00000890       ?BspESDHCCardDetectInt@CESDHCBase@@QAAXH@Z 10001890 f   bspesdhc.obj
 0001:000008f4       ?BspESDHCIsWriteProtected@CESDHCBase@@QAAHXZ 100018f4 f   bspesdhc.obj
 0001:00000944       ?BspGetRegistrySettings@CESDHCBase@@QAAHPAVCReg@@@Z 10001944 f   bspesdhc.obj
 0001:00000a38       ??0CESDHCBaseEDMA@@QAA@AAVCESDHCBase@@@Z 10001a38 f   bspesdhcdma.obj
 0001:00000a58       ?DmaSelectBit@CESDHCBaseEDMA@@UAAEXZ 10001a58 f i bspesdhcdma.obj
 0001:00000a60       ?BspEDMAInit@CESDHCBaseEDMA@@QAAHXZ 10001a60 f   bspesdhcdma.obj
 0001:00000a68       ?BspEDMAArm@CESDHCBaseEDMA@@QAAHAAU_SD_BUS_REQUEST@@H@Z 10001a68 f   bspesdhcdma.obj
 0001:00000a70       ?BspEDMANotifyEvent@CESDHCBaseEDMA@@QAAHAAU_SD_BUS_REQUEST@@W4_DMAEVENT@@@Z 10001a70 f   bspesdhcdma.obj
 0001:00000a78       ?BspEDMACheckCompletion@CESDHCBaseEDMA@@QAA?AW4_DMAEVENT@@H@Z 10001a78 f   bspesdhcdma.obj
 0001:00000a80       ??_GCESDHCBaseEDMA@@UAAPAXI@Z 10001a80 f i bspesdhcdma.obj
 0001:00000a80       ??_ECESDHCBaseEDMA@@UAAPAXI@Z 10001a80 f i bspesdhcdma.obj
 0001:00000ab0       DllEntry                   10001ab0 f   esdhcbase_common_topaz_v1:sdmain.obj
 0001:00000b04       SHC_Open                   10001b04 f   esdhcbase_common_topaz_v1:sdmain.obj
 0001:00000b08       SHC_Close                  10001b08 f   esdhcbase_common_topaz_v1:sdmain.obj
 0001:00000b10       SHC_PowerDown              10001b10 f   esdhcbase_common_topaz_v1:sdmain.obj
 0001:00000b20       SHC_PowerUp                10001b20 f   esdhcbase_common_topaz_v1:sdmain.obj
 0001:00000b50       SHC_IOControl              10001b50 f   esdhcbase_common_topaz_v1:sdmain.obj
 0001:00000b98       SHC_Deinit                 10001b98 f   esdhcbase_common_topaz_v1:sdmain.obj
 0001:00000bbc       SHC_Init                   10001bbc f   esdhcbase_common_topaz_v1:sdmain.obj
 0001:00000c24       ?IsDMACompleted@CESDHCBaseDMA@@UAA?AW4_DMAEVENT@@H@Z 10001c24 f i esdhcbase_common_topaz_v1:esdhc.obj
 0001:00000c38       ?DmaSelectBit@CESDHCBaseSDMA@@UAAEXZ 10001c38 f i esdhcbase_common_topaz_v1:esdhc.obj
 0001:00000c40       ??_ECESDHCBaseSDMA@@UAAPAXI@Z 10001c40 f i esdhcbase_common_topaz_v1:esdhc.obj
 0001:00000c40       ??_GCESDHCBaseSDMA@@UAAPAXI@Z 10001c40 f i esdhcbase_common_topaz_v1:esdhc.obj
 0001:00000c64       ??0CESDHCBase@@QAA@XZ      10001c64 f   esdhcbase_common_topaz_v1:esdhc.obj
 0001:00000cf0       ?SoftwareResetSDIO@CESDHCBase@@QAAXXZ 10001cf0 f   esdhcbase_common_topaz_v1:esdhc.obj
 0001:00000de0       ?SetClockRate@CESDHCBase@@QAAXPAK@Z 10001de0 f   esdhcbase_common_topaz_v1:esdhc.obj
 0001:00000f30       ?ClockGateOn@CESDHCBase@@QAAXXZ 10001f30 f   esdhcbase_common_topaz_v1:esdhc.obj
 0001:00000f48       ?ClockGateOff@CESDHCBase@@QAAXXZ 10001f48 f   esdhcbase_common_topaz_v1:esdhc.obj
 0001:00000f60       ?HandleInsertion@CESDHCBase@@QAAXXZ 10001f60 f   esdhcbase_common_topaz_v1:esdhc.obj
 0001:00001020       ??1CESDHCBase@@QAA@XZ      10002020 f   esdhcbase_common_topaz_v1:esdhc.obj
 0001:00001040       ?FreeHostContext@CESDHCBase@@QAAXHH@Z 10002040 f   esdhcbase_common_topaz_v1:esdhc.obj
 0001:000010b4       ?IOControl@CESDHCBase@@QAAHKPAEK0KPAK@Z 100020b4 f   esdhcbase_common_topaz_v1:esdhc.obj
 0001:000011ec       ?IndicateBusRequestComplete@CESDHCBase@@QAAXPAU_SD_BUS_REQUEST@@J@Z 100021ec f   esdhcbase_common_topaz_v1:esdhc.obj
 0001:0000129c       ?SDHCCancelIoHandler@CESDHCBase@@SAEPAU_SDCARD_HC_CONTEXT@@KPAU_SD_BUS_REQUEST@@@Z 1000229c f   esdhcbase_common_topaz_v1:esdhc.obj
 0001:000012a4       ?Open@CReg@@QAAHPAUHKEY__@@PBGK@Z 100022a4 f i esdhcbase_common_topaz_v1:esdhc.obj
 0001:0000130c       ?SetInterface@CESDHCBase@@QAAXPAU_SD_CARD_INTERFACE@@@Z 1000230c f   esdhcbase_common_topaz_v1:esdhc.obj
 0001:00001390       ?SendCommand@CESDHCBase@@QAAJPAU_SD_BUS_REQUEST@@@Z 10002390 f   esdhcbase_common_topaz_v1:esdhc.obj
 0001:000017c8       ?HandleRemoval@CESDHCBase@@QAAXH@Z 100027c8 f   esdhcbase_common_topaz_v1:esdhc.obj
 0001:000018e8       ?HandleCommandErrors@CESDHCBase@@QAAXXZ 100028e8 f   esdhcbase_common_topaz_v1:esdhc.obj
 0001:00001970       ?HandleDataErrors@CESDHCBase@@QAAXXZ 10002970 f   esdhcbase_common_topaz_v1:esdhc.obj
 0001:00001aa4       ?HandleReadReady@CESDHCBase@@QAAXXZ 10002aa4 f   esdhcbase_common_topaz_v1:esdhc.obj
 0001:00001c40       ?HandleWriteReady@CESDHCBase@@QAAXXZ 10002c40 f   esdhcbase_common_topaz_v1:esdhc.obj
 0001:00001dd4       ?HandleTransferComplete@CESDHCBase@@QAAXXZ 10002dd4 f   esdhcbase_common_topaz_v1:esdhc.obj
 0001:00001f80       ?Stop@CESDHCBase@@QAAJXZ   10002f80 f   esdhcbase_common_topaz_v1:esdhc.obj
 0001:000020ac       ?SlotOptionHandler@CESDHCBase@@QAAJW4_SD_SLOT_OPTION_CODE@@PAXK@Z 100030ac f   esdhcbase_common_topaz_v1:esdhc.obj
 0001:00002240       ?CommandCompleteHandler@CESDHCBase@@QAAHXZ 10003240 f   esdhcbase_common_topaz_v1:esdhc.obj
 0001:00002384       ?SDHCDeinitialize@CESDHCBase@@SAJPAU_SDCARD_HC_CONTEXT@@@Z 10003384 f   esdhcbase_common_topaz_v1:esdhc.obj
 0001:0000238c       ?SDHCSlotOptionHandler@CESDHCBase@@SAJPAU_SDCARD_HC_CONTEXT@@KW4_SD_SLOT_OPTION_CODE@@PAXK@Z 1000338c f   esdhcbase_common_topaz_v1:esdhc.obj
 0001:000023b0       ?HandleInterrupts@CESDHCBase@@QAAXXZ 100033b0 f   esdhcbase_common_topaz_v1:esdhc.obj
 0001:000026a4       ?ControllerIstThread@CESDHCBase@@QAAKXZ 100036a4 f   esdhcbase_common_topaz_v1:esdhc.obj
 0001:0000270c       ?BusRequestHandler@CESDHCBase@@QAAJPAU_SD_BUS_REQUEST@@@Z 1000370c f   esdhcbase_common_topaz_v1:esdhc.obj
 0001:0000280c       ?SDHCBusRequestHandler@CESDHCBase@@SAJPAU_SDCARD_HC_CONTEXT@@KPAU_SD_BUS_REQUEST@@@Z 1000380c f   esdhcbase_common_topaz_v1:esdhc.obj
 0001:00002818       ?ISTStub@CESDHCBase@@SAKPAX@Z 10003818 f i esdhcbase_common_topaz_v1:esdhc.obj
 0001:0000281c       ?Start@CESDHCBase@@QAAJXZ  1000381c f   esdhcbase_common_topaz_v1:esdhc.obj
 0001:00002a48       ?SDHCInitialize@CESDHCBase@@SAJPAU_SDCARD_HC_CONTEXT@@@Z 10003a48 f   esdhcbase_common_topaz_v1:esdhc.obj
 0001:00002a50       ?InterpretCapabilities@CESDHCBase@@QAAHXZ 10003a50 f   esdhcbase_common_topaz_v1:esdhc.obj
 0001:00002b10       ?Init@CESDHCBase@@QAAHPBG@Z 10003b10 f   esdhcbase_common_topaz_v1:esdhc.obj
 0001:00002c94       ??0CESDHCBaseDMA@@QAA@AAVCESDHCBase@@@Z 10003c94 f   esdhcbase_common_topaz_v1:esdhcdma.obj
 0001:00002d0c       ?Init@CESDHCBaseDMA@@UAAHXZ 10003d0c f   esdhcbase_common_topaz_v1:esdhcdma.obj
 0001:00002df8       ??1CESDHCBaseDMA@@UAA@XZ   10003df8 f   esdhcbase_common_topaz_v1:esdhcdma.obj
 0001:00002e84       ?ReAllocateDMABufferList@CESDHCBaseDMA@@QAAKK@Z 10003e84 f   esdhcbase_common_topaz_v1:esdhcdma.obj
 0001:00002eec       ?CancelDMA@CESDHCBaseDMA@@UAAHXZ 10003eec f   esdhcbase_common_topaz_v1:esdhcdma.obj
 0001:00002f3c       ?ArmDMA@CESDHCBaseDMA@@UAAHAAU_SD_BUS_REQUEST@@H@Z 10003f3c f   esdhcbase_common_topaz_v1:esdhcdma.obj
 0001:000030f8       ??1CESDHCBaseSDMA@@UAA@XZ  100040f8 f   esdhcbase_common_topaz_v1:esdhcdma.obj
 0001:00003134       ?Init@CESDHCBaseSDMA@@UAAHXZ 10004134 f   esdhcbase_common_topaz_v1:esdhcdma.obj
 0001:00003140       ?GetDMABuffer@CESDHCBaseSDMA@@IAAHAAU_SD_BUS_REQUEST@@H@Z 10004140 f   esdhcbase_common_topaz_v1:esdhcdma.obj
 0001:0000355c       ?ArmDMA@CESDHCBaseSDMA@@UAAHAAU_SD_BUS_REQUEST@@H@Z 1000455c f   esdhcbase_common_topaz_v1:esdhcdma.obj
 0001:000035c8       ?DMANotifyEvent@CESDHCBaseSDMA@@UAAHAAU_SD_BUS_REQUEST@@W4_DMAEVENT@@@Z 100045c8 f   esdhcbase_common_topaz_v1:esdhcdma.obj
 0001:000037d8       ?Init@CESDHCBaseEDMA@@UAAHXZ 100047d8 f   esdhcbase_common_topaz_v1:esdhcdma.obj
 0001:00003810       ?GetDMABuffer@CESDHCBaseEDMA@@IAAHAAU_SD_BUS_REQUEST@@H@Z 10004810 f   esdhcbase_common_topaz_v1:esdhcdma.obj
 0001:00003c40       ?ArmDMA@CESDHCBaseEDMA@@UAAHAAU_SD_BUS_REQUEST@@H@Z 10004c40 f   esdhcbase_common_topaz_v1:esdhcdma.obj
 0001:00003c90       ?DMANotifyEvent@CESDHCBaseEDMA@@UAAHAAU_SD_BUS_REQUEST@@W4_DMAEVENT@@@Z 10004c90 f   esdhcbase_common_topaz_v1:esdhcdma.obj
 0001:00003df4       ?IsDMACompleted@CESDHCBaseEDMA@@UAA?AW4_DMAEVENT@@H@Z 10004df4 f   esdhcbase_common_topaz_v1:esdhcdma.obj
 0001:00003e10       ??0CESDHCBase32BitADMA@@QAA@AAVCESDHCBase@@@Z 10004e10 f   esdhcbase_common_topaz_v1:esdhcdma.obj
 0001:00003e54       ?DmaSelectBit@CESDHCBase32BitADMA@@UAAEXZ 10004e54 f i esdhcbase_common_topaz_v1:esdhcdma.obj
 0001:00003e5c       ??1CESDHCBase32BitADMA@@UAA@XZ 10004e5c f   esdhcbase_common_topaz_v1:esdhcdma.obj
 0001:00003ee4       ?Init@CESDHCBase32BitADMA@@UAAHXZ 10004ee4 f   esdhcbase_common_topaz_v1:esdhcdma.obj
 0001:00003f74       ?GetDMABuffer@CESDHCBase32BitADMA@@QAAHAAU_SD_BUS_REQUEST@@H@Z 10004f74 f   esdhcbase_common_topaz_v1:esdhcdma.obj
 0001:00004418       ?ArmDMA@CESDHCBase32BitADMA@@UAAHAAU_SD_BUS_REQUEST@@H@Z 10005418 f   esdhcbase_common_topaz_v1:esdhcdma.obj
 0001:000045a8       ?DMANotifyEvent@CESDHCBase32BitADMA@@UAAHAAU_SD_BUS_REQUEST@@W4_DMAEVENT@@@Z 100055a8 f   esdhcbase_common_topaz_v1:esdhcdma.obj
 0001:000046ec       ??0CESDHCBase32BitADMA2@@QAA@AAVCESDHCBase@@@Z 100056ec f   esdhcbase_common_topaz_v1:esdhcdma.obj
 0001:00004730       ?DmaSelectBit@CESDHCBase32BitADMA2@@UAAEXZ 10005730 f i esdhcbase_common_topaz_v1:esdhcdma.obj
 0001:00004738       ??1CESDHCBase32BitADMA2@@UAA@XZ 10005738 f   esdhcbase_common_topaz_v1:esdhcdma.obj
 0001:000047c0       ?Init@CESDHCBase32BitADMA2@@UAAHXZ 100057c0 f   esdhcbase_common_topaz_v1:esdhcdma.obj
 0001:00004850       ?GetDMABuffer@CESDHCBase32BitADMA2@@QAAHAAU_SD_BUS_REQUEST@@H@Z 10005850 f   esdhcbase_common_topaz_v1:esdhcdma.obj
 0001:00004c60       ?IsEnoughDescTable@CESDHCBase32BitADMA2@@IAAHK@Z 10005c60 f   esdhcbase_common_topaz_v1:esdhcdma.obj
 0001:00004d24       ?DMANotifyEvent@CESDHCBase32BitADMA2@@UAAHAAU_SD_BUS_REQUEST@@W4_DMAEVENT@@@Z 10005d24 f   esdhcbase_common_topaz_v1:esdhcdma.obj
 0001:00004e30       ??_GCESDHCBaseDMA@@UAAPAXI@Z 10005e30 f i esdhcbase_common_topaz_v1:esdhcdma.obj
 0001:00004e30       ??_ECESDHCBaseDMA@@UAAPAXI@Z 10005e30 f i esdhcbase_common_topaz_v1:esdhcdma.obj
 0001:00004e54       ??_ECESDHCBase32BitADMA@@UAAPAXI@Z 10005e54 f i esdhcbase_common_topaz_v1:esdhcdma.obj
 0001:00004e54       ??_GCESDHCBase32BitADMA@@UAAPAXI@Z 10005e54 f i esdhcbase_common_topaz_v1:esdhcdma.obj
 0001:00004e78       ??_GCESDHCBase32BitADMA2@@UAAPAXI@Z 10005e78 f i esdhcbase_common_topaz_v1:esdhcdma.obj
 0001:00004e78       ??_ECESDHCBase32BitADMA2@@UAAPAXI@Z 10005e78 f i esdhcbase_common_topaz_v1:esdhcdma.obj
 0001:00004e9c       ?ArmDMA@CESDHCBase32BitADMA2@@UAAHAAU_SD_BUS_REQUEST@@H@Z 10005e9c f   esdhcbase_common_topaz_v1:esdhcdma.obj
 0001:00004fbc       ?CspESDHCGetBaseAddr@CESDHCBase@@QAAKK@Z 10005fbc f   esdhcbase_mx25_topaz_v1:mx25esdhc.obj
 0001:00004fe8       RegQueryValueExW           10005fe8 f   coredll:COREDLL.dll
 0001:00004ff8       KernelIoControl            10005ff8 f   coredll:COREDLL.dll
 0001:00005008       Sleep                      10006008 f   coredll:COREDLL.dll
 0001:00005018       SetInterruptEvent          10006018 f   coredll:COREDLL.dll
 0001:00005028       EventModify                10006028 f   coredll:COREDLL.dll
 0001:00005038       DisableThreadLibraryCalls  10006038 f   coredll:COREDLL.dll
 0001:00005048       SetLastError               10006048 f   coredll:COREDLL.dll
 0001:00005058       LocalFree                  10006058 f   coredll:COREDLL.dll
 0001:00005068       RegCloseKey                10006068 f   coredll:COREDLL.dll
 0001:00005078       CeSafeCopyMemory           10006078 f   coredll:COREDLL.dll
 0001:00005088       RegOpenKeyExW              10006088 f   coredll:COREDLL.dll
 0001:00005098       LocalAlloc                 10006098 f   coredll:COREDLL.dll
 0001:000050a8       CloseHandle                100060a8 f   coredll:COREDLL.dll
 0001:000050b8       WaitForSingleObject        100060b8 f   coredll:COREDLL.dll
 0001:000050c8       InterruptDisable           100060c8 f   coredll:COREDLL.dll
 0001:000050d8       LeaveCriticalSection       100060d8 f   coredll:COREDLL.dll
 0001:000050e8       EnterCriticalSection       100060e8 f   coredll:COREDLL.dll
 0001:000050f8       GetLastError               100060f8 f   coredll:COREDLL.dll
 0001:00005108       CreateEventW               10006108 f   coredll:COREDLL.dll
 0001:00005118       InterruptDone              10006118 f   coredll:COREDLL.dll
 0001:00005128       CeSetThreadPriority        10006128 f   coredll:COREDLL.dll
 0001:00005138       InterruptMask              10006138 f   coredll:COREDLL.dll
 0001:00005148       CreateThread               10006148 f   coredll:COREDLL.dll
 0001:00005158       InterruptInitialize        10006158 f   coredll:COREDLL.dll
 0001:00005168       OpenDeviceKey              10006168 f   coredll:COREDLL.dll
 0001:00005178       UnlockPages                10006178 f   coredll:COREDLL.dll
 0001:00005188       CacheRangeFlush            10006188 f   coredll:COREDLL.dll
 0001:00005198       LockPages                  10006198 f   coredll:COREDLL.dll
 0001:000051a8       MmUnmapIoSpace             100061a8 f   ceddk:CEDDK.dll
 0001:000051b8       OALDMAAllocBuffer          100061b8 f   ceddk:CEDDK.dll
 0001:000051c8       OALDMAFreeBuffer           100061c8 f   ceddk:CEDDK.dll
 0001:000051d8       MmMapIoSpace               100061d8 f   ceddk:CEDDK.dll
 0001:000051e8       DMACloseBuffer             100061e8 f   ceddk:CEDDK.dll
 0001:000051f8       DMAGetBufferPhysAddr       100061f8 f   ceddk:CEDDK.dll
 0001:00005208       DMAOpenBuffer              10006208 f   ceddk:CEDDK.dll
 0001:00005218       DDKClockGetFreq            10006218 f   cspddk:CSPDDK.dll
 0001:00005228       DDKGpioSetConfig           10006228 f   cspddk:CSPDDK.dll
 0001:00005238       DDKIomuxSelectInput        10006238 f   cspddk:CSPDDK.dll
 0001:00005248       DDKIomuxSetPadConfig       10006248 f   cspddk:CSPDDK.dll
 0001:00005258       DDKIomuxSetPinMux          10006258 f   cspddk:CSPDDK.dll
 0001:00005268       DDKClockSetGatingMode      10006268 f   cspddk:CSPDDK.dll
 0001:00005278       DDKGpioClearIntrPin        10006278 f   cspddk:CSPDDK.dll
 0001:00005288       DDKGpioReadDataPin         10006288 f   cspddk:CSPDDK.dll
 0001:00005298       DDKGpioReadIntrPin         10006298 f   cspddk:CSPDDK.dll
 0001:000052a8       ??3@YAXPAX@Z               100062a8 f   corelib1:COREDLL.dll
 0001:000052b8       ??2@YAPAXI@Z               100062b8 f   corelib1:COREDLL.dll
 0001:000052c8       __rt_udiv                  100062c8 f   corelib1:COREDLL.dll
 0001:000052d8       memset                     100062d8 f   corelib1:COREDLL.dll
 0001:000052e8       __C_specific_handler       100062e8 f   corelib1:COREDLL.dll
 0001:000052f8       wcsncpy_s                  100062f8 f   corelib1:COREDLL.dll
 0001:00005308       _purecall                  10006308 f   corelib1:COREDLL.dll
 0001:00005318       SDInitializeCardLib        10006318 f   sdcardlib:SDMemApi.obj
 0001:00005350       SDDeinitializeCardLib      10006350 f   sdcardlib:SDMemApi.obj
 0001:00005378       SDProcessException         10006378 f   sdcardlib:SDDebug.obj
 0001:0000539c       SDPerformSafeCopy          1000639c f   sdcardlib:SDDebug.obj
 0001:0000545c       svsutil_Initialize         1000645c f   sdcardlib:utilmem.obj
 0001:00005460       svsutil_DeInitialize       10006460 f   sdcardlib:utilmem.obj
 0001:00005464       svsutil_Alloc              10006464 f   sdcardlib:utilmem.obj
 0001:00005468       svsutil_ReAlloc            10006468 f   sdcardlib:utilmem.obj
 0001:0000546c       svsutil_Free               1000646c f   sdcardlib:utilmem.obj
 0001:00005470       SDHCDInitializeHCLib       10006470 f   sdhclib:SDHCLib.obj
 0001:00005488       SDHCDDeinitializeHCLib     10006488 f   sdhclib:SDHCLib.obj
 0001:00005490       SDHCDAllocateContext       10006490 f   sdhclib:SDHCLib.obj
 0001:000054bc       SDHCDDeleteContext         100064bc f   sdhclib:SDHCLib.obj
 0001:000054d4       SDHCDRegisterHostController 100064d4 f   sdhclib:SDHCLib.obj
 0001:000054ec       SDHCDDeregisterHostController 100064ec f   sdhclib:SDHCLib.obj
 0001:00005504       SDHCDIndicateSlotStateChange 10006504 f   sdhclib:SDHCLib.obj
 0001:0000551c       SDHCDIndicateBusRequestComplete 1000651c f   sdhclib:SDHCLib.obj
 0001:00005534       SDHCDGetAndLockCurrentRequest 10006534 f   sdhclib:SDHCLib.obj
 0001:0000554c       SDHCDGetHCFunctions        1000654c f   sdbus:SDBus.dll
 0001:0000555c       __security_check_cookie    1000655c f   corelib0:armsecgs.obj
 0001:0000556c       __gsfailure                1000656c     corelib0:armsecgs.obj
 0001:000055b0       memcpy                     100065b0 f   corelib1:COREDLL.dll
 0001:000055c0       malloc                     100065c0 f   corelib1:COREDLL.dll
 0001:000055d0       realloc                    100065d0 f   corelib1:COREDLL.dll
 0001:000055e0       free                       100065e0 f   corelib1:COREDLL.dll
 0001:000055f0       __report_gsfailure         100065f0 f   corelib1:COREDLL.dll
 0001:0000563c       __IMPORT_DESCRIPTOR_COREDLL 1000663c     coredll:COREDLL.dll
 0001:00005650       __IMPORT_DESCRIPTOR_CEDDK  10006650     ceddk:CEDDK.dll
 0001:00005664       __IMPORT_DESCRIPTOR_CSPDDK 10006664     cspddk:CSPDDK.dll
 0001:00005678       __IMPORT_DESCRIPTOR_SDBus  10006678     sdbus:SDBus.dll
 0001:0000568c       __NULL_IMPORT_DESCRIPTOR   1000668c     coredll:COREDLL.dll
 0002:00000000       __imp_DMAOpenBuffer        10007000     ceddk:CEDDK.dll
 0002:00000004       __imp_DMAGetBufferPhysAddr 10007004     ceddk:CEDDK.dll
 0002:00000008       __imp_DMACloseBuffer       10007008     ceddk:CEDDK.dll
 0002:0000000c       __imp_MmMapIoSpace         1000700c     ceddk:CEDDK.dll
 0002:00000010       __imp_OALDMAFreeBuffer     10007010     ceddk:CEDDK.dll
 0002:00000014       __imp_OALDMAAllocBuffer    10007014     ceddk:CEDDK.dll
 0002:00000018       __imp_MmUnmapIoSpace       10007018     ceddk:CEDDK.dll
 0002:0000001c       \177CEDDK_NULL_THUNK_DATA  1000701c     ceddk:CEDDK.dll
 0002:00000020       __imp_CloseHandle          10007020     coredll:COREDLL.dll
 0002:00000024       __imp_WaitForSingleObject  10007024     coredll:COREDLL.dll
 0002:00000028       __imp_InterruptDisable     10007028     coredll:COREDLL.dll
 0002:0000002c       __imp_LeaveCriticalSection 1000702c     coredll:COREDLL.dll
 0002:00000030       __imp_EnterCriticalSection 10007030     coredll:COREDLL.dll
 0002:00000034       __imp_GetLastError         10007034     coredll:COREDLL.dll
 0002:00000038       __imp_CreateEventW         10007038     coredll:COREDLL.dll
 0002:0000003c       __imp_InterruptDone        1000703c     coredll:COREDLL.dll
 0002:00000040       __imp_CeSetThreadPriority  10007040     coredll:COREDLL.dll
 0002:00000044       __imp_InterruptMask        10007044     coredll:COREDLL.dll
 0002:00000048       __imp_CreateThread         10007048     coredll:COREDLL.dll
 0002:0000004c       __imp_LocalAlloc           1000704c     coredll:COREDLL.dll
 0002:00000050       __imp_OpenDeviceKey        10007050     coredll:COREDLL.dll
 0002:00000054       __imp_UnlockPages          10007054     coredll:COREDLL.dll
 0002:00000058       __imp_CacheRangeFlush      10007058     coredll:COREDLL.dll
 0002:0000005c       __imp_LockPages            1000705c     coredll:COREDLL.dll
 0002:00000060       __imp_RegOpenKeyExW        10007060     coredll:COREDLL.dll
 0002:00000064       __imp_CeSafeCopyMemory     10007064     coredll:COREDLL.dll
 0002:00000068       __imp_RegCloseKey          10007068     coredll:COREDLL.dll
 0002:0000006c       __imp_LocalFree            1000706c     coredll:COREDLL.dll
 0002:00000070       __imp_SetLastError         10007070     coredll:COREDLL.dll
 0002:00000074       __imp_DisableThreadLibraryCalls 10007074     coredll:COREDLL.dll
 0002:00000078       __imp_RegQueryValueExW     10007078     coredll:COREDLL.dll
 0002:0000007c       __imp_EventModify          1000707c     coredll:COREDLL.dll
 0002:00000080       __imp_free                 10007080     corelib1:COREDLL.dll
 0002:00000084       __imp_realloc              10007084     corelib1:COREDLL.dll
 0002:00000088       __imp_malloc               10007088     corelib1:COREDLL.dll
 0002:0000008c       __imp_memcpy               1000708c     corelib1:COREDLL.dll
 0002:00000090       __imp_SetInterruptEvent    10007090     coredll:COREDLL.dll
 0002:00000094       __imp_Sleep                10007094     coredll:COREDLL.dll
 0002:00000098       __imp_KernelIoControl      10007098     coredll:COREDLL.dll
 0002:0000009c       __imp_InterruptInitialize  1000709c     coredll:COREDLL.dll
 0002:000000a0       __imp_??3@YAXPAX@Z         100070a0     corelib1:COREDLL.dll
 0002:000000a4       __imp_??2@YAPAXI@Z         100070a4     corelib1:COREDLL.dll
 0002:000000a8       __imp___rt_udiv            100070a8     corelib1:COREDLL.dll
 0002:000000ac       __imp_memset               100070ac     corelib1:COREDLL.dll
 0002:000000b0       __imp___C_specific_handler 100070b0     corelib1:COREDLL.dll
 0002:000000b4       __imp_wcsncpy_s            100070b4     corelib1:COREDLL.dll
 0002:000000b8       __imp__purecall            100070b8     corelib1:COREDLL.dll
 0002:000000bc       __imp___report_gsfailure   100070bc     corelib1:COREDLL.dll
 0002:000000c0       \177COREDLL_NULL_THUNK_DATA 100070c0     coredll:COREDLL.dll
 0002:000000c4       __imp_DDKClockGetFreq      100070c4     cspddk:CSPDDK.dll
 0002:000000c8       __imp_DDKGpioReadIntrPin   100070c8     cspddk:CSPDDK.dll
 0002:000000cc       __imp_DDKGpioReadDataPin   100070cc     cspddk:CSPDDK.dll
 0002:000000d0       __imp_DDKGpioClearIntrPin  100070d0     cspddk:CSPDDK.dll
 0002:000000d4       __imp_DDKClockSetGatingMode 100070d4     cspddk:CSPDDK.dll
 0002:000000d8       __imp_DDKIomuxSetPinMux    100070d8     cspddk:CSPDDK.dll
 0002:000000dc       __imp_DDKIomuxSetPadConfig 100070dc     cspddk:CSPDDK.dll
 0002:000000e0       __imp_DDKIomuxSelectInput  100070e0     cspddk:CSPDDK.dll
 0002:000000e4       __imp_DDKGpioSetConfig     100070e4     cspddk:CSPDDK.dll
 0002:000000e8       \177CSPDDK_NULL_THUNK_DATA 100070e8     cspddk:CSPDDK.dll
 0002:000000ec       __imp_SDHCDGetHCFunctions  100070ec     sdbus:SDBus.dll
 0002:000000f0       \177SDBus_NULL_THUNK_DATA  100070f0     sdbus:SDBus.dll
 0002:000000f8       g_SDClientApiFunctions     100070f8     sdcardlib:SDCardApiStubs.obj
 0002:0000012c       g_funcAlloc                1000712c     sdcardlib:utilmem.obj
 0002:00000130       g_funcFree                 10007130     sdcardlib:utilmem.obj
 0002:00000134       g_funcRealloc              10007134     sdcardlib:utilmem.obj
 0002:00000138       __security_cookie          10007138     corelib0:seccinit.obj
 0002:0000013c       __security_cookie_complement 1000713c     corelib0:seccinit.obj
 0002:0000014c       g_pvAllocData              1000714c     sdcardlib:utilmem.obj
 0002:00000150       g_pvFreeData               10007150     sdcardlib:utilmem.obj
 0002:00000154       ?g_pSDBusAccess@@3PAVSDBusAccess@@A 10007154     sdcardlib:busacc.obj

 entry point at        0001:00000ab0

 Static symbols

